:020000040800F2
:1000000060080020290100082501000825010008DA
:100010002501000825010008250100080000000056
:1000200000000000000000000000000025010008A2
:100030002501000800000000250100082501000836
:1000400025010008250100082501000825010008F8
:1000500025010008250100082501000825010008E8
:1000600025010008250100082501000825010008D8
:1000700025010008250100082501000825010008C8
:1000800025010008250100082501000800000000E6
:100090000000000000000000000000002501000832
:1000A0002501000825010008250100082501000898
:1000B000E908000861020008250100082501000880
:1000C0002501000825010008250100082501000878
:1000D00025010008B10800082501000825010008D5
:1000E0002501000825010008250100080000000086
:1000F0000000000000000000000000000000000000
:1001000000000000000000000000000000000000EF
:100110000000000000000000250100082501000883
:100120005FF808F1FEE700BF0C480D4A08B59042A1
:1001300007D2013A121A22F003020A49043204F0EB
:10014000A9FD094809494FF000028842B8BF40F8AC
:10015000042BFADBBDE8084000F020BE00000020C0
:10016000BC000020D4590008C0000020600400201A
:1001700030B5012185B0022001F0ACFE0021022043
:1001800001F0C0FE002505230E4C01A92046CDE953
:1001900001358DF80C5001F049FF2046012101F096
:1001A000C3FF01222046114601F0A4FF064B68461A
:1001B000009301F031FA2946204601F08DFF05B089
:1001C00030BD00BF000400401D00010110B5044611
:1001D00000210D4801F080FF21460B4801F096FFF9
:1001E0000021094801F090FF0121074801F074FF48
:1001F0000023064A13701378002BFCD0BDE8104092
:100200000021014801F068BF00040040C000002048
:1002100008B3F8B50027104C104D461E00212846A3
:1002200001F05AFF4FF47A71284601F06FFF002168
:10023000284601F069FF0121284601F04DFF277093
:100240002378002BFCD000212846013E01F044FF1A
:10025000731CE3D1F8BD7047C000002000040040CB
:1002600008B50121064801F053FF00B908BD01217E
:10027000034801F059FF0122024B1A7008BD00BF6C
:1002800000040040C0000020164991F800C04B78DF
:100290000CF10102D2B20A70C3B9012A19D000B51B
:1002A0000CF1FF3EBEF1060F07D80378023A134166
:1002B00003F0010318465DF804FBACF10802012AC3
:1002C00009D90B70022318465DF804FB013B4B7003
:1002D0000123184670470CF1020C012381F800C07D
:1002E000E8E700BFC1000020F0B520271F4E83B013
:1002F000002205460C461E4840F22551C6F884707F
:1003000001F080FF40F22551194801F0C5FF4FF47C
:100310005871174801F0C0FF0021154801F064FF33
:1003200001214FF4804001F0C9FD00234FF4402229
:1003300010490F484B608A608B810D6001F0F8FE18
:100340000D4B01A8019301F067F90121084801F064
:100350004BFF0CB903B0F0BD012240F22551044817
:1003600001F050FF776003B0F0BD00BF00E100E096
:1003700000380140C8000020250F020100214FF085
:10038000006001F07FB900BF10B501F0A7FC4FF489
:10039000803001F0C7FC01F0E1FC012800D010BD65
:1003A0000446102001F0F6FA022001F0E9FA90204C
:1003B00001F0FEFC4FF4A06001F00EFD4FF48060F0
:1003C00001F000FD204601F0E1FC01F0E9FC042809
:1003D000FBD110BD2DE9F047904C0121042001F024
:1003E0006DFD21468E4B8F4841F8103F01F0DEFA3B
:1003F0000121082001F062FD21468B4B8B4841F81A
:10040000103F01F0D3FA214604274FF4804A884B6D
:10041000864841F8103F01F0C9FA844804F1100100
:10042000E774A4F810A001F0C1FA0121102001F036
:1004300045FD21467F4B804841F8103F01F0B6FA58
:1004400021467E4B794841F8103F01F0AFFA504603
:10045000012101F03FFD4FF08273636118230025F5
:100460004FF4006923620723754804F11401A38443
:10047000C4F81890A58301F087FD0121704801F0B0
:10048000C1FD01216E4801F0A9FD4FF482736C4853
:1004900004F11401E38201F077FD2146694B6148C4
:1004A00041F8103F01F082FA4FF480635D4804F197
:1004B00010012382E77401F079FA29464FF41650AF
:1004C000FFF712FF2146604B584841F8103F01F0FA
:1004D0006DFA564804F11001E774A4F8109001F089
:1004E00065FA8022594B2946C3F88420584801F008
:1004F0007BFE01214FF4802001F0ECFC4FF4964389
:100500004FF4402221465248A2602360A5816560D5
:1005100001F00EFE01214E4801F066FE0121022687
:10052000084601F0BFFC4B4801F06AF904F1540899
:1005300001214948C4E90C562565C4F82C8001F016
:10054000E9F8464B0022A3628023C4E90E234FF44E
:1005500080724FF48063C4E9102320224FF40053CB
:100560003C4804F12801C4E9122301F0DDF901211E
:10057000384801F0F9F940232A4804F11001238298
:10058000E57401F013FA20232146264821F8103F94
:10059000E57401F00BFA284601F028FC01214FF424
:1005A000007001F08BFC40F201174FF46022002331
:1005B000294804F15801C4E91823A56584F8686046
:1005C000A4F85C7001F076F803230122052122488B
:1005D00001F0C8F80323324606211F4801F0C2F893
:1005E00001211D4801F096F81B48012101F088F80F
:1005F000194801F099F8184801F09CF80028FAD140
:10060000154801F09BF8144801F09EF80028FAD133
:10061000BDE8F0470121104801F09AB8C800002059
:10062000001001100008014080010110000C014081
:1006300000A00118002001100010014000800118E6
:1006400000380040000201180004011800E100E039
:100650000048004008000240002401404C240140B2
:1006600070B5184C184B2146184841F8103F01F05E
:100670009DF901214FF4804001F02CFC4FF0827273
:100680004FF400630021C4E9052307231822104D0D
:1006900004F114062846A1833146A384226201F0A6
:1006A00073FC2846012101F0ADFC2846012101F030
:1006B00095FC4FF4827331462846E382BDE87040D2
:1006C00001F062BCC800002000800118000C01404D
:1006D0000038004008B5064801F020FC054B0649EB
:1006E000064841F8103FBDE8084001F05FB900BF7F
:1006F0000038004000800110C8000020000C0140BC
:10070000012130B5044685B0084601F0E3FB002125
:10071000012001F0F7FB144B002293FBF4F30525B5
:10072000013B01A94FF08040ADF80830ADF80A2038
:100730008DF80C20019501F079FC01214FF08040EB
:1007400001F0F2FC01224FF08040114601F0D2FC92
:10075000064B6846009300F05FFF01214FF0804098
:1007600001F0BAFC05B030BD40420F001C00010191
:10077000F8B51446002A00F08F8000EBD0704010CE
:100780000E4603F0BFF8454903F0C4F9444903F0AD
:1007900005F84449074603F0BDF903F0CDFAC5B2A8
:1007A000284603F0AFF83F4903F000F90146384608
:1007B00002F0F2FF41352570074603F0BDFAC5B2DD
:1007C000284603F09FF80146384602F0E5FF303531
:1007D0003549A570054603F09DF903F0ADFAC0B2A6
:1007E00000F14103237103F08DF82F4903F0DEF887
:1007F0000146284602F0D0FF2C4903F08BF903F0A4
:100800009BFA03463033A371304603F07BF823494B
:1008100003F080F9224902F0C1FF2249064603F0A5
:1008200079F903F089FAC5B2284603F06BF81D493F
:1008300003F0BCF80146304602F0AEFF413565706A
:10084000064603F079FAC5B2284603F05BF8014684
:10085000304602F0A1FF30351349E570054603F03C
:1008600059F903F069FAC0B200F14103637103F072
:1008700049F80D4903F09AF80146284602F08CFF2A
:100880000A4903F047F903F057FA034600223033D0
:10089000E37122720120F8BD1046F8BD8096184B16
:1008A0000000B44200002041ABAA2A3D8988883B61
:1008B00008B540F225510B4801F0CCFC38B109488D
:1008C00001F0BEFCBDE80840C0B202F075B84FF4BC
:1008D0005871044801F0BEFCBDE80840014801F031
:1008E000AFBC00BF0038014070B501214FF080401F
:1008F00001F00EFC00B970BD01214FF0804001F005
:1009000013FC02F02BFB00284DD1594E594D738832
:100910002A689BB29342584C31DCA378002B74D1E7
:100920000023238023889BB25BB9708880B202F0D9
:100930009DFE4DA3D3E9002302F01CFC02F000FF52
:100940002860E378002B32D1E37843B9E368013BB8
:10095000E36023B901232374E368013BE360AB68E0
:10096000013BAB60002BC6D1637C002B3AD02B79C6
:10097000002B45D100236374C823AB6070BD23886E
:1009800001339BB2238023889BB2192BCAD9012340
:100990004FF480713948A37001F09CF980213748E9
:1009A00001F098F9BEE7BDE8704002F0D1BA606886
:1009B000FFF76AFCA3782072002BC5D102282AD049
:1009C00001283AD00028BFD101460122732000F04F
:1009D0005DFC2B79002BB7D04FF48071274801F0D4
:1009E0007BF9B1E7A37C1B0602D401236374C3E740
:1009F0002B79002BF9D08021204801F06BF9F4E726
:100A000080211E4801F068F9B4E74FF480511C487A
:100A100001F060F984E72B79F3B963685A1C6260CE
:100A20005B7803F0FF02002B8ED14FF4C073E270AD
:100A3000E360227400F010FD86E702460221732075
:100A400000F024FC2B79002B3FF47EAF4FF4807133
:100A50000A4801F03FF977E74FF48071074801F049
:100A600039F9DAE7AFF300809A9999999999F13FAA
:100A70001C0100200000002034010020000C014077
:100A80000008014028222DE9F04FAE4B85B01A70C6
:100A900000F07AFD4FF416720146AB4BAB4C1B884D
:100AA00004F118009BB202FB03F31B13E174A38251
:100AB00001F0DEFCD4E9061094F82C30A44A022B95
:100AC000A37CA44D8CBF43F0800303F07F03A37489
:100AD000FFF74EFEA769A04AE66982FB073182FB59
:100AE00006324FEAE778C8EBA1584FEAE679002FC3
:100AF0009A49C9EBA252B8BF7F42B8F1000FB8BF04
:100B0000C8F1000882EAE279002E01FB0877A9EB20
:100B1000E279B8BF764201FB0966002F636C904A08
:100B20009049B8BF7F422846002EB8BF764204F0F5
:100B3000C7F894F82930834694F82B208A4900930B
:100B4000281894F82A3004F0BBF8DFF820A288496E
:100B5000AAFB06C6AAFB07C7B609CDE90296854AD5
:100B60000BEB0006E069BF09009712EA200738BFC7
:100B70000F46A069019712EA200238BF0A46434691
:100B80007D49A81904F09CF8236A06448AFB032ACD
:100B9000DB17C3EBAA127949A81904F091F80644AF
:100BA000626A7649A81904F08BF806447449A5F1E5
:100BB0001402A81904F084F8064494F9132071492A
:100BC000A81904F07DF86FF06301A38A6E4A064409
:100BD000A2FB0372520901FB0233A8196B4904F00E
:100BE0006FF8064494F828206649A81904F068F8BC
:100BF000A37C37180093E28D238E6549E81904F031
:100C00005FF894F84C603844002E00F096804FF660
:100C1000FF7341F22102291D43E05B001FFA83FCB0
:100C20001BB2002B49DB4FEA4C0C1FFA8CF30FFA76
:100C30008CFCBCF1000F48DB4FEA430C1FFA8CF32D
:100C40000FFA8CFCBCF1000F47DB4FEA430C1FFA94
:100C50008CF30FFA8CFCBCF1000F46DB4FEA430C1F
:100C60001FFA8CF30FFA8CFCBCF1000F45DB4FEA46
:100C7000430C1FFA8CF30FFA8CFCBCF1000F44DB21
:100C80004FEA430C1FFA8CF30FFA8CFCBCF1000FF7
:100C900011F8016FACBF5B0082EA43039BB2002EE8
:100CA00039D083EA06231E04B7D582EA430C0FFA33
:100CB0008CF3002B1FFA8CFCB5DA82EA4C030FFA96
:100CC00083FCBCF1000F9BB2B6DA82EA43030FFA51
:100CD00083FCBCF1000F9BB2B7DA82EA43030FFA40
:100CE00083FCBCF1000F9BB2B8DA82EA43030FFA2F
:100CF00083FCBCF1000F9BB2B9DA82EA43030FFA1E
:100D000083FCBCF1000F9BB2BADA82EA43030FFA0C
:100D100083FC9BB2BAE71A461E4928448B831E49BE
:100D200003F0CEFF656000F0E3FB0122636CE2702C
:100D30001344636405B0BDE8F08F4FF6FF721346AD
:100D4000EAE700BFC20000201C010020340100209F
:100D5000680100207C0100206BCA5F6B806967FF1F
:100D60000C000020DC550008E8550008D34D621047
:100D7000DC5600085C560008F855000810560008BC
:100D8000185600081C5600081F85EB512056000815
:100D90002C56000800000020385600082DE9F04FBE
:100DA00087B0FFF7F1FAFFF7E9FAFFF713FB4B20E3
:100DB000FFF7A6FCFFF7DCF901F074FB764B1B791B
:100DC000002B40F0E2800C21744801F035FA00F06D
:100DD00069FB734800F088FA012205216D2000F0BC
:100DE00055FA01220021712000F050FA0122F02171
:100DF000132000F04BFA01220021122000F046FAE5
:100E0000012280210F2000F041FA00220123654CCD
:100E1000032504F14801E27061602374022602F0A8
:100E20007DF8DFF884A1DFF8848104F1180704F16C
:100E30003409E3786BB9237C5BB186B1013D013E97
:100E400015F0FF05F6B24ED0FFF71CFEE378002B3D
:100E5000F1D00021102000F01FFC30BFE9E700F0C6
:100E600047FB00F091FB4FF41672BAF80030E074C3
:100E70009BB202FB03F338461B13A38201F0F8FA7E
:100E8000D4E9061094F82C304A46022BA37C8CBF80
:100E900043F0800303F07F03A374FFF769FC002194
:100EA000404601F0A1F9A28A94F91330CDE903324A
:100EB0003F4B93E807008DE8070097E80F0002F02A
:100EC00053F80121404601F08FF900F0C5FAE378AC
:100ED000002B53D1237C002B50D0013D15F0FF0592
:100EE0004FF00106B0D1257400F04EFB4FF416729E
:100EF000BAF80030E0749BB202FB03F338461B13D0
:100F0000A38201F0B5FAD4E9061094F82C304A46D1
:100F1000022BA37CDFF89CB08CBF43F0800303F06E
:100F20007F03A374FFF724FC234B032593E80700FA
:100F3000ABE8030021498BF800205846ABF11C02B6
:100F400003F0BEFE034601221D49ABF1080EB1F8C5
:100F500000C0083389782EF803C073449970732059
:100F6000114600F093F9ABF1080000F02DF84FF4B2
:100F7000FA60FFF74DF90123237465E70021102083
:100F8000022600F089FB30BF53E74FF480710D4813
:100F900000F0A0FE17E700BF00000020004800405E
:100FA00000C0D843340100201C010020003801405B
:100FB0005C0100207C010020405600084C560008CF
:100FC00054560008000C0140F8B50478002C4AD0B3
:100FD0000646A64FA4F16103DAB2192A25D9A4F175
:100FE0004103DAB2192A46D9A4F13003DAB2092A48
:100FF0005DD9A4F12B03152B76D8DFE813F004019B
:10100000ED007500D700C000750075007500750013
:101010007500750075007500750075007500750028
:101020007500A800750091007A0057F823502C78BD
:1010300054B911E02D2C1AD000F080FA3C20FFF7B3
:10104000E7F815F8014F3CB100F052FA2E2CF1D11F
:101050003C20FFF7DDF8EFE7B420FFF7D9F816F8EA
:10106000014F002CB6D1BDE8F84000F0F5B9B4202E
:10107000FFF7CEF8E0E757F823502C785CB9EBE7A0
:101080002D2C10D000F05AFA3C20FFF7C1F815F8CB
:10109000014F002CE0D000F02BFA2E2CF0D13C2098
:1010A000FFF7B6F8EEE7B420FFF7B2F8EAE707EB90
:1010B00083039D6E2C785CB9CEE72D2C10D000F008
:1010C0003DFA3C20FFF7A4F815F8014F002CC3D0DF
:1010D00000F00EFA2E2CF0D13C20FFF799F8EEE745
:1010E000B420FFF795F8EAE74FF4D270FFF790F8D5
:1010F000B5E72E245E4D0BE02D2C00F0A38000F010
:101100001DFA3C20FFF784F815F8014F002CA3D0FE
:1011100000F0EEF92E2CEFD13C20FFF779F8EEE746
:101120002E24544D0BE02D2C00F0888000F006FAA0
:101130003C20FFF76DF815F8014F002C8CD000F023
:10114000D7F92E2CEFD13C20FFF762F8EEE72D24E3
:10115000494D0CE02D2C00F0858000F0EFF93C208B
:10116000FFF756F815F8014F002C3FF475AF00F06B
:10117000BFF92E2CEED13C20FFF74AF8EDE72D24E5
:101180003E4D0BE02D2C69D000F0D8F93C20FFF744
:101190003FF815F8014F002C3FF45EAF00F0A8F9BE
:1011A0002E2CEFD13C20FFF733F8EDE7344D0BE068
:1011B0002D2C4FD000F0C2F93C20FFF729F815F88C
:1011C000014F002C3FF448AF00F092F92E2CEFD1E4
:1011D0003C20FFF71DF8EDE72D242A4D0BE02D2CC8
:1011E00034D000F0ABF93C20FFF712F815F8014FAE
:1011F000002C3FF431AF00F07BF92E2CEFD13C20D6
:10120000FFF706F8EDE72E241F4D0BE02D2C11D033
:1012100000F094F93C20FEF7FBFF15F8014F002C7D
:101220003FF41AAF00F064F92E2CEFD13C20FEF70A
:10123000EFFFEDE7B420FEF7EBFFE9E7B420FEF7A0
:10124000E7FF73E7B420FEF7E3FF58E7B420FEF7AB
:10125000DFFFC6E7B420FEF7DBFFABE7B420FEF705
:10126000D7FF91E7B420FEF7D3FF76E738570008A1
:10127000F8570008E8570008D0570008C85700087A
:10128000D8570008E0570008F057000810B522B3FF
:1012900040F08000000204B20C4311484FF40051AA
:1012A000A4B200F019FD02210E4800F0B9FE00289A
:1012B000F9D021460B4800F09FFE0121094800F0BB
:1012C000AFFE0028F9D04FF40051054800F002FDB0
:1012D000044800F093FEC0B210BD000204B2DBE788
:1012E0000010014000380040F8B55349074602F0AD
:1012F0005DFB5249054602F00BFD06465049003E93
:10130000284618BF012602F005FC02F015FD4B49E6
:101310000446284602F0FCFC0346002B14BF6FF085
:1013200017030023751CE4B22846183C1C4402F045
:10133000E9FA444902F03AFB0146384602F0EAFB7A
:1013400094FBF5F40546E0B202F0DCFA01462846CB
:1013500002F022FA3C4902F01FFA3C4902F026FB57
:1013600002F0EAFC054604F01F0444EA461444F483
:1013700075444FF40051364844F04004ADB200F0DB
:10138000ABFC0221334800F04BFE0028F9D0214687
:10139000304800F031FE01212E4800F041FE0028C7
:1013A000F9D04FF400512A4800F094FC294800F08D
:1013B00025FE2C0A4FF40051254844F4764400F0F1
:1013C0008BFC0221234800F02BFE0028F9D0214697
:1013D000204800F011FE01211E4800F021FE0028E7
:1013E000F9D04FF400511A4800F074FC194800F08D
:1013F00005FEEDB24FF40051154845F4774500F075
:101400006BFC0221134800F00BFE0028F9D029469E
:10141000104800F0F1FD01210E4800F001FE002807
:10142000F9D00B484FF4005100F054FCBDE8F840EF
:10143000084800F0E3BD00BF3BB1933F0000F0431C
:1014400000002041ABAA0A410000C04100007A47D9
:1014500000100140003800404FF4005108B50F481B
:1014600000F03AFC02210E4800F0DAFD0028F9D025
:1014700048F240710A4800F0BFFD0121084800F021
:10148000CFFD0028F9D005484FF4005100F022FCB0
:10149000BDE80840024800F0B1BD00BF00100140A7
:1014A000003800404FF4005108B50F4800F014FC1C
:1014B00002210E4800F0B4FD0028F9D048F28071F6
:1014C0000A4800F099FD0121084800F0A9FD002814
:1014D000F9D005484FF4005100F0FCFBBDE808408E
:1014E000024800F08BBD00BF0010014000380040F2
:1014F0004FF4005108B50F4800F0EEFB02210E48F2
:1015000000F08EFD0028F9D048F24B710A4800F037
:1015100073FD0121084800F083FD0028F9D005483B
:101520004FF4005100F0D6FBBDE80840024800F03F
:1015300065BD00BF00100140003800404FF400516D
:1015400008B50F4800F0C8FB02210E4800F068FD06
:101550000028F9D048F243710A4800F04DFD0121FE
:10156000084800F05DFD0028F9D005484FF400510F
:1015700000F0B0FBBDE80840024800F03FBD00BFEE
:1015800000100140003800404FF4005110B52048D1
:1015900000F0A2FB02211F4800F042FD0028F9D014
:1015A00041F2FF111B4800F027FD0121194800F00E
:1015B00037FD0028F9D04FF40051154800F08AFBA0
:1015C000144800F01BFD0446C4F34604503C4FF49D
:1015D00000510F4864B200F07FFB02210D4800F07B
:1015E0001FFD0028F9D048F680710A4800F004FD7C
:1015F0000121084800F014FD0028F9D04FF40051F3
:10160000034800F067FB034800F0F8FC204610BDDB
:101610000010014000380040C37813B3174A30B5BA
:10162000D1684FF0010EC9430F23827890F801C0B2
:101630000078C1F3022100F01F040EFA04F4CB403D
:10164000C1F1040E13400CFA0EFC0D4D43EA0C03DD
:101650001B012A18DBB2400982F8003345F820400C
:1016600030BD0121037806485A0903F01F032032D8
:1016700001FA03F340F82230704700BF00ED00E0AC
:1016800000E100E021F06041024B21F07F010143C5
:101690009960704700ED00E021B1054B1A691043D5
:1016A00018617047024A136923EA0000106170470D
:1016B00000ED00E0436891F804C023F4702310B4F7
:1016C00023F480730C6843EA0C232343436083684C
:1016D0000A4A91F805C01A40D1E902432343134353
:1016E00043EA4C0383600A7CC36A013A23F4700323
:1016F000D2B243EA025310BCC3627047FDF7F1FF58
:10170000836819B143F001038360704723F001033C
:1017100083607047836819B143F4807383607047B6
:1017200023F4807383607047836843F00803836009
:10173000704700BF8068C0F3C0007047836843F003
:1017400004038360704700BF8068C0F38000704767
:10175000836819B143F4A0038360704723F4A003A6
:1017600083607047092910B52FD94FF0070EA1F1FA
:101770000A0CC4680CEB4C0C03FA0CF30EFA0CFCCC
:1017800024EA0C0C43EA0C03C360062A4FF01F0C3A
:101790000CD8013A446B02EB820201FA02F30CFA14
:1017A00002F224EA02021343436310BD0C2A1AD842
:1017B000073A046B02EB820201FA02F30CFA02F21E
:1017C00024EA02021343036310BD4FF0070C0469BF
:1017D00001EB410E0CFA0EFC03FA0EF324EA0C04A2
:1017E00023430361D1E70D3AC46A02EB820201FA96
:1017F00002F30CFA02F224EA02021343C36210BDA0
:101800004FF6FE7C00230268394902EA0C02884246
:101810000260036043608360C36027D0354B984209
:101820001ED0354B98422DD0344B984230D0344B9B
:10183000984221D0334B984230D0334B984239D024
:10184000324B98423CD0324B98422DD0314B98428B
:101850003CD0314B98423FD0304B984242D07047F9
:101860002F4A536843F0F003536070472C4A536883
:1018700043F00F0353607047294A536843F47023C1
:1018800053607047264A536843F47063536070474F
:10189000234A536843F4704353607047204A5368A7
:1018A00043F47003536070471E4A536843F0F003DB
:1018B000536070471A4A536843F07063536070472F
:1018C000184A536843F00F0353607047154A536832
:1018D00043F4706353607047124A536843F4704393
:1018E000536070470F4A536843F470235360B6E760
:1018F000080002401C000240300002404400024048
:10190000580002406C00024080000240080402407F
:101910001C040240300402404404024058040240C7
:1019200000000240000402408B6810B40C6A0A698F
:1019300023431343D1E9052413432343CC690268AD
:1019400023434C6A22F4FF4223438C6A22F0700244
:101950002343CC6813430360D1E9002344608260D1
:1019600010BCC360704700BF21B1036843F001039E
:10197000036070474FF6FE720368134003607047C0
:10198000034A136803F0380303431360704700BF32
:1019900000200240044B196821F0100119601A68F8
:1019A00002431A60704700BF0020024000B591F862
:1019B00003C01CF0100F18BF8B780CF00F0E18BF6F
:1019C0004EEA030E0B88DAB2002A36D0BCF1480F7B
:1019D000026800F0B380BCF1280F00F03A81D9070B
:1019E00044BF22F00F024EEA0202990744BF22F0E0
:1019F000F00242EA0E12590744BF22F4706242EA32
:101A00000E22190744BF22F4704242EA0E32D90670
:101A100044BF22F4702242EA0E42990644BF22F4E7
:101A2000700242EA0E52590644BF22F0706242EA46
:101A30000E62190600F10A810260FF2B4AD9BCF13F
:101A4000480F426848D1D90506D54FF4807122F07D
:101A50000F024EEA02020161990506D54FF40071AA
:101A600022F0F00242EA0E120161590506D54FF448
:101A7000806122F4706242EA0E220161190506D5E6
:101A80004FF4006122F4704242EA0E320161D9043F
:101A900006D54FF4805122F4702242EA0E420161D1
:101AA000990406D54FF4005122F4700242EA0E5216
:101AB0000161590406D54FF4804122F0706242EA78
:101AC0000E6201611B0404D54FF400436EF31F72D4
:101AD000036142605DF804FBBCF1280F6ED0D905AC
:101AE00044BF22F00F024EEA0202990544BF22F0E1
:101AF000F00242EA0E12590544BF22F4706242EA33
:101B00000E22190544BF22F4704242EA0E32D90473
:101B100044BF22F4702242EA0E42990444BF22F4E8
:101B2000700242EA0E52590444BF22F0706242EA47
:101B30000E621B04CDD56EF31F72CAE7D90705D517
:101B4000012122F00F024EEA02020161990705D538
:101B5000022122F0F00242EA0E120161590705D576
:101B6000042122F4706242EA0E220161190705D5B0
:101B7000082122F4704242EA0E320161D90605D5ED
:101B8000102122F4702242EA0E420161990605D525
:101B9000202122F4700242EA0E520161590605D555
:101BA000402122F0706242EA0E62016119067FF55F
:101BB00043AF80216EF31F7201613DE7D90506D561
:101BC0004FF4807122F00F024EEA02024161990542
:101BD00006D54FF4007122F0F00242EA0E12416184
:101BE000590506D54FF4806122F4706242EA0E2254
:101BF0004161190506D54FF4006122F4704242EAB2
:101C00000E324161D90406D54FF4805122F470227E
:101C100042EA0E424161990406D54FF4005122F484
:101C2000700242EA0E524161590406D54FF48041D8
:101C300022F0706242EA0E6241611B047FF549AFF7
:101C40004FF400436EF31F72436142E76EF31F725D
:101C5000F2E6D90705D5012122F00F024EEA020271
:101C60004161990705D5022122F0F00242EA0E12E5
:101C70004161590705D5042122F4706242EA0E221F
:101C80004161190705D5082122F4704242EA0E325B
:101C90004161D90605D5102122F4702242EA0E4294
:101CA0004161990605D5202122F4700242EA0E52C4
:101CB0004161590605D5402122F0706242EA0E6268
:101CC000416119067FF5B8AE80216EF31F72416144
:101CD000B2E600BF016170474161704710B4002057
:101CE0004FF41F040D4B0E4A196841F001011960B1
:101CF00059680A405A601A6822F0847222F48032CD
:101D00001A601A6822F480221A605A6822F4FE02CD
:101D10005A609C6010BCD862704700BF001002403F
:101D20000000FFF80C4BB0F5803F1A6822F48032B7
:101D30001A601A6822F480221A6008D0B0F5802F49
:101D400004D11A6842F4A0221A60704770471A68DA
:101D500042F480321A60704700100240002382B0C3
:101D60000949019300E04AB90A68019B02F4003274
:101D700001330193019BB3F5A06FF4D1024B1868B6
:101D8000C0F3404002B0704700100240034A53685D
:101D900023F0030303435360704700BF0010024069
:101DA000024B586800F00C00704700BF0010024062
:101DB000034A536823F0F00303435360704700BFA6
:101DC00000100240034A536823F4E0630343536066
:101DD000704700BF00100240034A536823F4605369
:101DE00043EAC0035360704700100240034A53683F
:101DF00023F4404303435360704700BF0010024088
:101E0000234A10B4536803F00C03042B24D0082B8E
:101E100026D0204A134602601D491F4A4C68C4F36D
:101E20000314145DE34043604C68C4F30224145D62
:101E300023FA04F484604C68C4F3C22C12F80C40FA
:101E4000E340C360496810BCC1F381310A44127C8D
:101E5000B3FBF2F303617047104A13460260DBE7FD
:101E600053685168C3F38343C90303F1020304D4E5
:101E70000B4A02FB03F30360CEE7D26A074902F084
:101E80000F020132B1FBF2F202FB03F30360C3E77E
:101E90000010024000127A004400002000366E015B
:101EA00000093D00044A536911B11843506170475D
:101EB00023EA00005061704700100240044A936911
:101EC00011B118439061704723EA00009061704798
:101ED00000100240044AD36911B11843D061704721
:101EE00023EA0000D061704700100240044AD36822
:101EF00011B11843D060704723EA0000D0607047EA
:101F000000100240044A136911B118431061704770
:101F100023EA0000106170470010024008B5174B1B
:101F2000984206D0164B98420FD0164B984218D0C4
:101F300008BD01214FF48050FFF7D8FFBDE80840ED
:101F400000214FF48050FFF7D1BF01214FF48040B2
:101F5000FFF7D8FFBDE8084000214FF48040FFF7AD
:101F6000D1BF01214FF40040FFF7CCFFBDE808408E
:101F700000214FF40040FFF7C5BF00BF0030014013
:101F800000380040003C0040B1F802C00B888A884D
:101F900043EA0C03B1F806C013430A8943EA0C0371
:101FA00000B5B1F80AE0B1F80CC0134343EA0E03E0
:101FB000028843EA0C03B1F80EC002F4415243EA2E
:101FC0000C0313439BB20380838B0A8A23F40063C0
:101FD0001B041B0C838302825DF804FB038821B180
:101FE0009BB243F040030380704723F040031B047F
:101FF0001B0C0380704700BF81817047808980B2CD
:10200000704700BF838821B19BB243F004038380F3
:10201000704723F004031B041B0C8380704700BF30
:102020000389194214BF012000207047274A038802
:1020300090429BB212D002F5006290420ED0B0F1F5
:10204000804F0BD0A2F59832904207D002F5806203
:10205000904203D002F58062904203D14A8823F077
:10206000700313431A4A904217D002F580629042DF
:1020700013D0CA8823F440739BB21343B1F804C051
:102080000380124B0A889842A0F82CC002850CD11C
:102090000B7A038601238382704703808B888385B4
:1020A0000B8803850123838270470A4B9842EFD047
:1020B00003F540639842EBD003F580639842E7D084
:1020C00003F580639842E3D0ECE700BF002C0140A9
:1020D0000010004000340140038821B19BB243F05E
:1020E00001030380704723F001031B041B0C0380D2
:1020F000704700BF83899BB212B119438181704739
:1021000023EA01018181704781847047818570478E
:10211000038A828911EA030092B203D00A4214BFF3
:1021200001200020704700BFC94389B20182704777
:1021300030B504460D46238ACA889BB223F4405327
:1021400013438A892382A389898823F4B05323F017
:102150000C031B041B0C0B43298987B00B436989B3
:1021600001A80B439BB2A381A38A9BB223F44073C3
:102170001343A382FFF744FEDDE9033218491948EF
:102180008C4208BF1346A28903EB830312F4004F6D
:102190002A6803EB830314BF52009200B3FBF2F3EF
:1021A0006425A0FB0321490905FB11330A01A1891C
:1021B00009040AD41B013233A0FB0313C3F34313F6
:1021C00013439BB2238107B030BDDB003233A0FB49
:1021D0000313C3F3421313439BB2238107B030BDF3
:1021E000003801401F85EB51838921B19BB243F434
:1021F00000538381704723F400531B041B0C83811D
:10220000704700BF012301F01F0CC1F342110129E7
:1022100003FA0CF30DD002290CBF103014301AB1A0
:102220000268134303607047026822EA03030360F5
:1022300070470C30F3E700BFC1F30801818070479D
:102240008088C0F3080070470388194214BF01203A
:10225000002070470123C1F3421201F01F0C012A34
:1022600003FA0CF313D0022A0CBF028A828A92B2BC
:102270001340028892B243B10123090A03FA01F123
:102280000A4214BF184600207047184670478289DA
:1022900092B21340EDE700BF0123090A8B40DB43F4
:1022A0009BB20380704700BF044A05491368002BA6
:1022B00008BF0B46184410601846704744020020BF
:1022C00060040020FEE700002DE9F84F984643180F
:1022D000DBB2174603EB0802D2B2C518154402EB75
:1022E0001822D6B2354481468A46EDB24FEA182B01
:1022F000B8F1000F0AD000243B5D01341E44F6B251
:10230000E3B2354498451C46EDB2F5D8574C402110
:102310002046FFF799FF0028F9D0B5215348FFF771
:102320008BFF524C40212046FFF78EFF0028F9D04A
:102330004E4C40212046FFF787FF0028F9D062214C
:102340004A48FFF779FF494C40212046FFF77CFFC0
:102350000028F9D0454C40212046FFF775FF0028A2
:10236000F9D049464148FFF767FF404C40212046DD
:10237000FFF76AFF0028F9D03C4C40212046FFF7C8
:1023800063FF0028F9D051463848FFF755FF374C16
:1023900040212046FFF758FF0028F9D0334C402158
:1023A0002046FFF751FF0028F9D041462F48FFF79C
:1023B00043FF2E4C40212046FFF746FF0028F9D06E
:1023C0002A4C40212046FFF73FFF0028F9D059460C
:1023D0002648FFF731FF254C40212046FFF734FF08
:1023E0000028F9D0B8F1000F1AD008F1FF339BB2E2
:1023F0001E4C07F1FF381F4418F8019F402120466A
:10240000FFF722FF0028F9D049462046FFF714FFC6
:1024100040212046FFF718FF0028F9D04745EBD1AF
:10242000124C40212046FFF70FFF0028F9D031461B
:102430000E48FFF701FF0D4C40212046FFF704FF37
:102440000028F9D0094C40212046FFF7FDFE002866
:10245000F9D029460548FFF7EFFE044C40212046FD
:10246000FFF7F2FE0028F9D0BDE8F88F00380140F0
:1024700010B4844672B60A4C0FCCCCF80000CCF8ED
:102480000410CCF80820CCF80C3007CCCCF81000A5
:10249000CCF81410CCF8182062B610BC704700BFFE
:1024A000480200202DE9F0430124FFB05A22002108
:1024B00003A802F0FDFBBC4ABC4B21464FF416407A
:1024C000019202938DF80C40FDF70EFF0A20FDF7F4
:1024D0009FFEBDF808300DF10A029DF807109DF827
:1024E0000600FFF7F1FE4FF44870FDF791FE21461C
:1024F0004FF41650FDF7F8FE0A20FDF789FEBDF8EF
:1025000008309DF807100DF10A029DF80600FFF74C
:10251000DBFE4FF44870FDF77BFE622200211AA813
:1025200002F0C6FB4FF40C614FF4164200230DF18C
:102530006D06ADF872104FF00111ADF87620402510
:1025400032464FF01A089A48ADF87430ADF878303A
:10255000984B1A900DF181071B93CDF87A1012F861
:10256000013F43445FFA83F845449742EDB2F6D108
:10257000914C40212046FFF767FE0028F9D0B52195
:102580008D48FFF759FE8C4C40212046FFF75CFE3A
:102590000028F9D0884C40212046FFF755FE00283E
:1025A000F9D062218448FFF747FE834C4021204642
:1025B000FFF74AFE0028F9D07F4C40212046FFF764
:1025C00043FE0028F9D006217B48FFF735FE7A4C00
:1025D00040212046FFF738FE0028F9D0764C4021F4
:1025E0002046FFF731FE0028F9D000217248FFF79E
:1025F00023FE714C40212046FFF726FE0028F9D02B
:102600006D4C40212046FFF71FFE0028F9D0142111
:102610006948FFF711FE684C40212046FFF714FE81
:102620000028F9D0644C40212046FFF70DFE002819
:10263000F9D000216048FFF7FFFD5F4C40212046A4
:10264000FFF702FE0028F9D05B4C16F8019F4021ED
:102650002046FFF7F9FD0028F9D049462046FFF74C
:10266000EBFD40212046FFF7EFFD0028F9D0B742EF
:10267000EBD1514C40212046FFF7E6FD0028F9D070
:1026800041464D48FFF7D8FD4B4C40212046FFF70F
:10269000DBFD0028F9D0484C40212046FFF7D4FD4F
:1026A0000028F9D029464448FFF7C6FD424C402196
:1026B0002046FFF7C9FD0028F9D001214FF416404C
:1026C000FDF712FE0A20FDF7A3FD3C4B3C4800211C
:1026D000CDE933035A2235A802F0EAFA0026022394
:1026E00011210620374C0DF1D202FFF7EDFDC9256F
:1026F0002677667708E0637F4BB90120FDF788FDF8
:102700006B1E13F0FF0502D0237F002BF3D0237F35
:1027100033B99DF8CE009DF8CF10BDF8D030E2E778
:102720005A2200214EA802F0C3FA0322264B0121AF
:1027300040F201254C93062000261346ADF83421C3
:10274000ADF836518DF838110DF59B72FFF7BCFDD1
:10275000C9252677667708E0637F4BB90120FDF72E
:1027600057FD6B1E13F0FF0502D0237F002BF3D023
:10277000237F33B99DF832019DF83311BDF8343110
:10278000E2E7062300268DF83731BDF834319DF895
:1027900033119DF832010DF59B72FFF795FDC925A8
:1027A000267766771BE000BFB56206040400FFFFD2
:1027B000B562060014000100003801400200080460
:1027C000B562061148020020B5620601637F4BB96D
:1027D0000120FDF71DFD6B1E13F0FF0502D0237FC6
:1027E000002BF3D0237F002BCFD0212300268DF8A0
:1027F0003731BDF834319DF833119DF832010DF5B4
:102800009B72FFF761FDC9252677667708E0637F35
:102810004BB90120FDF7FCFC6B1E13F0FF0502D045
:10282000237F002BF3D0237F002BE2D05A220021FC
:1028300067A802F03DFA40F2072142F210721C48EC
:10284000242365900220ADF89C11ADF8A22105214A
:102850004FF019128DF8B10116480026CDE96A2013
:102860008DF8A61106201946134AADF8A4616692A8
:102870000DF5CD72FFF728FDC9252677667708E0AC
:10288000637F4BB90120FDF7C3FC6B1E13F0FF05FE
:1028900002D0237F002BF3D0237F33B99DF896011C
:1028A0009DF89711BDF89831E2E77FB0BDE8F0835D
:1028B000B562062464002C012400FF03F0B590F8F3
:1028C00002E0C57884880EEB0502D2B21119C9B2B4
:1028D00072440A4401EB1421CFB23A44861DD2B2AD
:1028E0005CB10023F15C013339445FFA83FCCFB261
:1028F0003A4464456346D2B2F4D8315D3319B942E3
:1029000004D02C4A138B01331383F0BD5B789342C0
:10291000F7D1BEF1010F0AD0BEF1050FF5D1012D9F
:1029200045D0002DF1D10122224B5A77F0BD072D61
:102930000DD0022D26D0062D32D0212DE5D11D4BF4
:10294000847DC17D027EDC7499745A74F0BD194B8C
:10295000817EDA8A19750132DA82D0F82240D0F805
:102960001E10D0F82A20C3E90041817B9A60D974F7
:10297000C17B427F9974017CD0F8424059741A742B
:10298000DC60F0BD0B4BD0F81610DA8A0132DA8227
:10299000D0F80A40D0F80E209960C3E90024F0BDB9
:1029A000044B017C90F8352019751A74F0BD014B69
:1029B0001D77F0BD4802002010B51A4CA37F83B9E3
:1029C000E37F23B9B52820D00023E37710BD012B86
:1029D000FAD16228F8D10222A37784F82100E277A5
:1029E00010BDE37FE218042B82F8200004D9A28CEA
:1029F000591E083291420DD00133DBB2632B89BFDF
:102A00000023E377E377A37710BD012384F8200048
:102A1000E37710BD04F12000FFF750FF0023E377B8
:102A2000A37710BD48020020A1F17E03B3FA83F31F
:102A30002DE9F04700262D4C5B0940F289174FF035
:102A40000108894605466670237012E0BAF1000F4E
:102A50003BD084F802800121B5F87001FDF7B6FB88
:102A600063784FEA59090133DBB2072B63703AD818
:102A7000237809F0010A002BE8D12B8883EA0A02A7
:102A8000D1074FEA530344BF83F4044383F00803A0
:102A90002B80BAF1000F18D0A3780133DBB2052BDD
:102AA000A370D8D10121B5F87001FDF78FFB95F81F
:102AB0006931A670022B16BF4FF0020A3B46CA23AB
:102AC00085F869A1A5F86E31C5E795F86931A6705A
:102AD000022B15BF02220122CA233B4685F8692139
:102AE000A5F86E31B7E7BDE8F08700BFD00200203F
:102AF000F8B5044641480D461746FEF7F5FB01229E
:102B000005217220FEF7C2FB4FF400513C48FFF74D
:102B1000E1F8012212217120FEF7B8FBFDF7DAFD82
:102B20000123B4F8040184F86C31002863D194F8CF
:102B30006B31002B56D000234FF40041314884F80C
:102B40006B31FFF7C9F84FF08042002601214FF6A4
:102B5000FF70138823F001031B041B0C1380B4F8CF
:102B60006E319385968413889BB20B431380A378B0
:102B7000208084F8691143B17E212046FFF754FF7D
:102B80000136A178F3B29942F6D83FB12F4415F837
:102B9000011B2046FFF748FFBD42F8D123880025DE
:102BA000D9436FEA1323184E2046C9B2F370FFF7DA
:102BB0003BFF2046F178FFF737FF7E212046FFF7E5
:102BC00033FFFDF74DFD114884F86C51FEF78CFB87
:102BD000012229467120FEF759FB4B20FDF790FD9D
:102BE0002846F8BD01234FF40041064884F86B31B4
:102BF000FFF770F8A7E7FDF70BFB98E70040D84315
:102C000000100140000C0140D002002000C0D84359
:102C10002DE9F04F4FF0203904469A46904683B094
:102C20009DF83020061D0192C0F80B900622DDE9C8
:102C30000DB7A0F80F900B300F9D02F071F85146C0
:102C40000622C4F804903046A6F8049002F068F812
:102C5000B8F1400F88BFA8F10608019B88BF5FFA52
:102C600088F8A37284F81180584602F051F8804623
:102C7000594608F1010204F1120002F00BF800239A
:102C80005FFA88F808F10E00E1180A790133DBB227
:102C9000520083420A71F7D34FF0030C3946F027F4
:102CA00008F10D0323441A79204442F001021A71FD
:102CB00080F804C004EB080308F110002A46DF7412
:102CC000304402F02DF83146204605F1100242440E
:102CD00003B0BDE8F04FFFF70BBF00BF70B504466F
:102CE00084B008460D4602F013F8064694F81331F6
:102CF00004F58A71029594F80C212046CDE9003143
:102D0000039604F20D1304F58371FFF781FF04B0FD
:102D100070BD00BFF8B508460D46144601F0F8FF37
:102D200010F0FF0059D04FF0000C6A1E63462025BA
:102D3000461E0FE02D2908BF2021664550D003F123
:102D4000010EE1545FFA8EF30CF1010C5FFA8CF185
:102D5000814241D212F8011F2C29EBD1062B44D815
:102D6000C3F10701C9B203F1010E0129E5545FFA6D
:102D70008EFE29D004F80E50022903F1020E5FFAEC
:102D80008EFE21D004F80E50032903F1030E5FFAE2
:102D90008EFE19D004F80E50042903F1040E5FFAD8
:102DA0008EFE11D004F80E5003F1050E5FFA8EF777
:102DB000A1F1050E1EF0FF0E06D0E5559F1DFFB2D6
:102DC000BEF1010F18BFE5550CF1010C0B445FFA81
:102DD0008CF18142DBB2BDD31C4400232370F8BDCB
:102DE0005F1CE154FBB2062BBAD9A3F108010529F7
:102DF00003D8C3F10E01C9B2B5E7A3F10F0105294C
:102E0000A2D8C3F11501C9B2ADE700BF2DE9F04F5B
:102E100083B09DF838404FF0190E01274FF000089D
:102E2000019404461E464FF02035DFF88CC0DFF8D1
:102E30008CB0C0F86EC1CBF8040080F8681180F83F
:102E400002E0C270A0F8047180F86A719DF830A0A9
:102E5000DDF83490DDF83CB0FDF702FC184884F84A
:102E60006C81FEF741FA3A4641467120FEF70EFAB0
:102E70004B20FDF745FC3146C4F80651A4F80A5131
:102E800004F5837001F03CFF494684F80CA1C4F8B6
:102E90000D51A4F8115104F20D1001F031FF594603
:102EA0002046019B04F58A7284F8133103B0BDE813
:102EB000F04FFFF72FBF00BF89011B03D002002096
:102EC00000C0D84310B590F86B310446D3B100234D
:102ED0004FF40041104884F86B31FEF7FDFE4FF0CF
:102EE00080420021138823F001031B041B0C138074
:102EF000B4F86E319385918413889BB243F001033B
:102F0000138010BD01234FF40041034884F86B3156
:102F1000FEF7E0FEE3E700BF000C014010B5002221
:102F2000302442210648074B84B00390019300915E
:102F3000054B114605480294FFF768FF04B010BD29
:102F40000C5800081C58000804580008D80200203B
:102F50000148FFF7B7BF00BFD8020020014B93F82C
:102F60006C017047D802002084B02DE9F041AEB06A
:102F700034AC84E80F00764B092883FB00234FEA2A
:102F8000E0729DF9EC40BDF8F050C2EBA30340F3B2
:102F900095807049704E81FB0010C2EBA0506F4AC3
:102FA00040B202FB0033C3EB03139B0086FB0326F6
:102FB0006B4A82FB0312D917C1EBA643C1EB223146
:102FC00003EB8302C3EBC20201EB8201C9B2359E5F
:102FD0005F4A4FEAE67C82FB0672092ECCEBA20226
:102FE00040F38E805B4F87FB0676CCEBA65C5B4E96
:102FF0004FFA8CFC06FB0C22574EC2EB02129200D9
:1030000086FB0276564F87FB02E7D217C2EBA64635
:10301000C2EB273206EB8607C6EBC70702EB870237
:10302000D2B205922F22002800910292C8BF4E21F1
:1030300080EAE072D8BF5321BCF1000FA2EBE0722E
:10304000CCBF4520572006904F20F6B204964FF48F
:103050004D66CDE90B458CEAEC74A4EBEC74E4B25C
:103060000394369D3F4C0790E81784FB0575C0EB31
:10307000A51006FB00F084FB0054C017C0EBA410A1
:10308000394C01910890B4F87401DBB2013080B280
:103090000990A4F874019DF8E000D2B20A90334878
:1030A00033490D900EA801F00BFE20460EA9FFF744
:1030B00015FE2EB0BDE8F04104B07047264E5842D0
:1030C000A6FB0020254F40F3874207FB02F2D31AEC
:1030D000C3EB03139A00224986FB026381FB026162
:1030E000D217C2EBA343C2EB213203EB8301800C66
:1030F000C3EBC101404202EB810140B2C9B266E7B5
:10310000154EC2F1000CA6FB0C7CDFF850804CF38E
:10311000874E08FB0EFEAEEB0202C2EB02129200DB
:103120000F4F86FB02E687FB02E7D217C2EBA646EB
:10313000C2EB273206EB86074FEA9C4CC6EBC7076B
:10314000CCF1000C02EB87024FFA8CFCD2B268E79C
:10315000676666666BCA5F6B83DE1B43C0BDF0FFAC
:10316000AD8BDB68D34D6210D80200207058000888
:103170003458000870B54FF0FF0C4CF4E06C1CEABA
:1031800011541DBF1CEA135594EA0C0F95EA0C0F5D
:1031900000F0DEF82C4481EA030621EA4C5123EAD0
:1031A0004C5350EA013518BF52EA033541F48011FF
:1031B00043F4801338D0A0FB02CE4FF00005E1FBB2
:1031C00002E506F00042E0FB03E54FF00006E1FBFC
:1031D00003569CF0000F18BF4EF0010EA4F1FF043F
:1031E000B6F5007F64F5407404D25FEA4E0E6D417F
:1031F00046EB060642EAC62141EA55514FEAC52090
:1032000040EA5E504FEACE2EB4F1FD0C88BFBCF50B
:10321000E06F1ED8BEF1004F08BF5FEA500E50F1BC
:10322000000041EB045170BD06F0004646EA010182
:1032300040EA020081EA0301B4EB5C04C2BFD4EBB4
:103240000C0541EA045170BD41F480114FF0000EAD
:10325000013C00F3AB8014F1360FDEBF002001F01B
:10326000004170BDC4F10004203C35DA0C341BDC95
:1032700004F11404C4F1200500FA05F320FA04F067
:1032800001FA05F240EA020001F0004221F000419B
:1032900010EBD37021FA04F642EB06015EEA430E0E
:1032A00008BF20EAD37070BDC4F10C04C4F120053E
:1032B00000FA04F320FA05F001FA04F240EA0200F1
:1032C00001F0004110EBD37041F100015EEA430EC2
:1032D00008BF20EAD37070BDC4F1200500FA05F2E2
:1032E0004EEA020E20FA04F301FA05F243EA020361
:1032F00021FA04F001F0004121FA04F220EA020070
:1033000000EBD3705EEA430E08BF20EAD37070BDB5
:1033100094F0000F0FD101F00046400041EB010195
:1033200011F4801F08BF013CF7D041EA060195F077
:10333000000F18BF704703F00046520043EB030331
:1033400013F4801F08BF013DF7D043EA060370471E
:1033500094EA0C0F0CEA135518BF95EA0C0F0CD029
:1033600050EA410618BF52EA4306D1D181EA03016F
:1033700001F000414FF0000070BD50EA410606BF69
:103380001046194652EA430619D094EA0C0F02D1AE
:1033900050EA013613D195EA0C0F05D152EA0336F3
:1033A0001CBF104619460AD181EA030101F0004111
:1033B00041F0FE4141F470014FF0000070BD41F05A
:1033C000FE4141F4780170BD81F0004102E000BF90
:1033D00083F0004330B54FEA41044FEA430594EAD5
:1033E000050F08BF90EA020F1FBF54EA000C55EA10
:1033F000020C7FEA645C7FEA655C00F0E2804FEAE1
:103400005454D4EB5555B8BF6D420CDD2C4480EAC2
:10341000020281EA030382EA000083EA010180EAF2
:10342000020281EA0303362D88BF30BD11F0004F40
:103430004FEA01314FF4801C4CEA113102D0404276
:1034400061EB410113F0004F4FEA03334CEA1333B1
:1034500002D0524263EB430394EA050F00F0A780C9
:10346000A4F10104D5F1200E0DDB02FA0EFC22FAC4
:1034700005F2801841F1000103FA0EF2801843FAB8
:1034800005F359410EE0A5F120050EF1200E012AA9
:1034900003FA0EFC28BF4CF0020C43FA05F3C018E7
:1034A00051EBE37101F0004507D54FF0000EDCF160
:1034B000000C7EEB00006EEB0101B1F5801F1BD309
:1034C000B1F5001F0CD349085FEA30004FEA3C0C0D
:1034D00004F101044FEA445212F5800F80F09A8003
:1034E000BCF1004F08BF5FEA500C50F1000041EB07
:1034F000045141EA050130BD5FEA4C0C404141EB0B
:103500000101013C28BFB1F5801FE9D291F0000F05
:1035100004BF01460020B1FA81F308BF2033A3F1B4
:103520000B03B3F120020CDA0C3208DD02F1140CAB
:10353000C2F10C0201FA0CF021FA02F10CE002F1E6
:103540001402D8BFC2F1200C01FA02F120FA0CFCDF
:10355000DCBF41EA0C019040E41AA2BF01EB045128
:10356000294330BD6FEA04041F3C1CDA0C340EDC26
:1035700004F11404C4F1200220FA04F001FA02F369
:1035800040EA030021FA04F345EA030130BDC4F127
:103590000C04C4F1200220FA02F001FA04F340EA1C
:1035A0000300294630BD21FA04F0294630BD94F0CD
:1035B000000F83F4801306BF81F480110134013DB4
:1035C0004EE77FEA645C18BF7FEA655C29D094EA25
:1035D000050F08BF90EA020F05D054EA000C04BFA3
:1035E0001946104630BD91EA030F1EBF002100208E
:1035F00030BD5FEA545C05D14000494128BF41F02D
:10360000004130BD14F580043CBF01F5801130BD90
:1036100001F0004545F0FE4141F470014FF000001B
:1036200030BD7FEA645C1ABF194610467FEA655CCC
:103630001CBF0B46024650EA013406BF52EA03356E
:1036400091EA030F41F4002130BD00BF90F0000F5C
:1036500004BF0021704730B54FF4806404F1320498
:103660004FF000054FF0000150E700BF90F0000F51
:1036700004BF0021704730B54FF4806404F1320478
:1036800010F0004548BF40424FF000013EE700BF48
:1036900042004FEAE2014FEA31014FEA02701FBFD8
:1036A00012F07F4393F07F4F81F06051704732F00A
:1036B0007F4208BF704793F07F4F04BF41F4002161
:1036C000704730B54FF4607401F0004521F00041BF
:1036D0001CE700BF50EA010208BF704730B54FF049
:1036E00000050AE050EA010208BF704730B511F04A
:1036F000004502D5404261EB41014FF4806404F182
:1037000032045FEA915C3FF4D8AE4FF003025FEA07
:10371000DC0C18BF03325FEADC0C18BF033202EB8B
:10372000DC02C2F1200300FA03FC20FA02F001FAE5
:1037300003FE40EA0E0021FA02F11444BDE600BF88
:103740004FEA410212F5001215D211D56FF47873C9
:10375000B3EB625212D94FEAC12343F0004343EA6C
:10376000505311F0004F23FA02F018BF4042704747
:103770004FF00000704750EA013005D111F00040D1
:1037800008BF6FF0004070474FF00000704700BF67
:1037900080F0004002E000BF81F0004142001FBF06
:1037A0005FEA410392EA030F7FEA226C7FEA236C0F
:1037B0006AD04FEA1262D2EB1363C1BFD218414004
:1037C00048404140B8BF5B42192B88BF704710F09A
:1037D000004F40F4000020F07F4018BF404211F03D
:1037E000004F41F4000121F07F4118BF494292EAA5
:1037F000030F3FD0A2F1010241FA03FC10EB0C00D1
:10380000C3F1200301FA03F100F0004302D549425D
:1038100060EB4000B0F5000F13D3B0F1807F06D30A
:1038200040084FEA310102F10102FE2A51D2B1F102
:10383000004F40EBC25008BF20F0010040EA0300F7
:103840007047490040EB0000013A28BFB0F5000F77
:10385000EDD2B0FA80FCACF1080CB2EB0C0200FA2D
:103860000CF0AABF00EBC25052421843BCBFD0407C
:103870001843704792F0000F81F4000106BF80F4F6
:1038800000000132013BB5E74FEA41037FEA226CB9
:1038900018BF7FEA236C21D092EA030F04D092F084
:1038A000000F08BF0846704790EA010F1CBF0020B8
:1038B000704712F07F4F04D1400028BF40F0004015
:1038C000704712F100723CBF00F50000704700F035
:1038D000004343F0FE4040F4000070477FEA22625C
:1038E00016BF08467FEA23630146420206BF5FEA2D
:1038F000412390EA010F40F4800070474FF000032D
:1039000004E000BF10F0004348BF40425FEA000CF3
:1039100008BF704743F0964301464FF000001CE09B
:1039200050EA010208BF70474FF000030AE000BFF1
:1039300050EA010208BF704711F0004302D540422F
:1039400061EB41015FEA010C02BF844601460020A1
:1039500043F0B64308BFA3F18053A3F50003BCFABC
:103960008CF2083AA3EBC25310DB01FA02FC634469
:1039700000FA02FCC2F12002BCF1004F20FA02F270
:1039800043EB020008BF20F00100704702F1200263
:1039900001FA02FCC2F1200250EA4C0021FA02F2C4
:1039A00043EB020008BF20EADC7070474FF0FF0CC9
:1039B0001CEAD0521EBF1CEAD15392EA0C0F93EAC4
:1039C0000C0F6FD01A4480EA010C400218BF5FEA66
:1039D00041211ED04FF0006343EA501043EA5111D9
:1039E000A0FB01310CF00040B1F5000F3EBF4900D3
:1039F00041EAD3715B0040EA010062F17F02FD2AD7
:103A00001DD8B3F1004F40EBC25008BF20F00100B9
:103A1000704790F0000F0CF0004C08BF49024CEAD0
:103A2000502040EA51207F3AC2BFD2F1FF0340EA62
:103A3000C250704740F400004FF00003013A5DDCD3
:103A400012F1190FDCBF00F000407047C2F1000214
:103A5000410021FA02F1C2F1200200FA02FC5FEA01
:103A6000310040F1000053EA4C0308BF20EADC704B
:103A7000704792F0000F00F0004C02BF400010F4BD
:103A8000000F013AF9D040EA0C0093F0000F01F06A
:103A9000004C02BF490011F4000F013BF9D041EA8C
:103AA0000C018FE70CEAD15392EA0C0F18BF93EA8E
:103AB0000C0F0AD030F0004C18BF31F0004CD8D1B8
:103AC00080EA010000F00040704790F0000F17BF3F
:103AD00090F0004F084691F0000F91F0004F14D085
:103AE00092EA0C0F01D142020FD193EA0C0F03D1DD
:103AF0004B0218BF084608D180EA010000F00040E0
:103B000040F0FE4040F40000704740F0FE4040F4BA
:103B1000400070474FF0FF0C1CEAD0521EBF1CEA59
:103B2000D15392EA0C0F93EA0C0F69D0A2EB030277
:103B300080EA010C49024FEA402037D04FF0805311
:103B400043EA111143EA10130CF000408B4238BFD6
:103B50005B0042F17D024FF4000C8B4224BF5B1AE4
:103B600040EA0C00B3EB510F24BFA3EB510340EA32
:103B70005C00B3EB910F24BFA3EB910340EA9C00E0
:103B8000B3EBD10F24BFA3EBD10340EADC001B0150
:103B900018BF5FEA1C1CE0D1FD2A3FF650AF8B42F4
:103BA00040EBC25008BF20F0010070470CF0004C01
:103BB0004CEA50207F32C2BFD2F1FF0340EAC2502C
:103BC000704740F400004FF00003013A37E792F0ED
:103BD000000F00F0004C02BF400010F4000F013A4B
:103BE000F9D040EA0C0093F0000F01F0004C02BF46
:103BF000490011F4000F013BF9D041EA0C0195E7AF
:103C00000CEAD15392EA0C0F08D142027FF47DAF47
:103C100093EA0C0F7FF470AF084676E793EA0C0F37
:103C200004D14B023FF44CAF08466EE730F0004C35
:103C300018BF31F0004CCAD130F000427FF45CAFC5
:103C400031F000437FF43CAF5FE700BF4FF0FF3C33
:103C500006E000BF4FF0010C02E000BF4FF0010C86
:103C60004DF804CD4FEA40024FEA41037FEA226C4F
:103C700018BF7FEA236C11D001B052EA530C18BF71
:103C800090EA010F58BFB2EB030088BFC81738BFD6
:103C90006FEAE17018BF40F0010070477FEA226CC4
:103CA00002D15FEA402C05D17FEA236CE4D15FEAC0
:103CB000412CE1D05DF8040B704700BF84460846F4
:103CC0006146FFE70FB5FFF7C9FF002848BF10F1B5
:103CD000000F0FBD4DF808EDFFF7F4FF0CBF0120FA
:103CE00000205DF808FB00BF4DF808EDFFF7EAFF84
:103CF00034BF012000205DF808FB00BF4DF808ED3F
:103D0000FFF7E0FF94BF012000205DF808FB00BF33
:103D10004DF808EDFFF7D2FF94BF012000205DF8B9
:103D200008FB00BF4DF808EDFFF7C8FF34BF0120C6
:103D300000205DF808FB00BF42000ED2B2F1FE4F3A
:103D40000BD34FF09E03B3EB126209D44FEA00236A
:103D500043F0004323FA02F070474FF00000704731
:103D600012F1610F01D1420202D14FF0FF307047D2
:103D70004FF00000704700BF03685A004CBF43F08B
:103D8000004323F000431844704700BF2DE9F84377
:103D900039B34F1E044615463E464FF0000808EB67
:103DA000060101EBD171491004EBC1094846FFF748
:103DB000E3FF0346C80008308F4220440BD0AB42DB
:103DC0000BD8FFF7D9FF0138A84201F10108E6D36B
:103DD0004846BDE8F883AB42FAD9884501D04E1E6B
:103DE000DDE74FF000094846BDE8F883012807D019
:103DF000022807D0044B00280CBF1846002070474B
:103E00000248704702487047DD440008E14400085A
:103E1000E544000830B5244B044683B08D1E3BB307
:103E2000284601A9AFF30080E8B101992A46FFF7BF
:103E3000ADFF0146B8B1FFF79FFF4B68A064012BAF
:103E40002ED0002B27DB081DFFF796FF0023C4E9C7
:103E500013030368002B12DBFFF78EFF03460020DD
:103E6000236103B030BD00230920236103B030BDBE
:103E70000E4B0F491846C91AC9100191D6E7C3F372
:103E80000360FFF7B3FF0028034614BF002009209A
:103E9000236103B030BD0123081DC4E91303D8E733
:103EA000002305202361DCE700000000CC58000857
:103EB000D4590008036810B5DA07044606D49B07F6
:103EC00000F1480009D500F05DFC2368590709D5C9
:103ED0001A070ED5DB0613D510BD00F04BFC236886
:103EE0005907F5D404F1D00000F054FC23681A07F8
:103EF000F0D404F5A87000F055FC2368DB06EBD481
:103F000004F5E870BDE8104000F090BC092070474F
:103F10000346006800B11844704700BF704700BFF7
:103F200070B504460E462046316CFFF773FF054618
:103F300098B9D6F840C03246214601202369C4F81A
:103F400014C098470828EED0072806D12846316CBF
:103F5000FFF7E4FF301D00F001FCFEF7B3F900BFEE
:103F60002DE9F0474FF0000AADF5727D0DF10C0E12
:103F700001F1040CC768D0F8188006461446BCE866
:103F80000F00AEE80F00BCE80F00AEE80F00BCE881
:103F90000F00AEE80F009CE80F0002AD8EE80F00A6
:103FA000C5F800A021E02B6C4FF4F0722946736134
:103FB0007AA800F06FFE3146504633697AAA9847D6
:103FC000889C82466C643346324649460120CDE9DE
:103FD0000058B8470446F0B94FF4F07228467AA961
:103FE00000F058FEBAF1080F1BD13046296CFFF7DC
:103FF00011FF04F109095FFA89FA04460028D2D0BA
:10400000A96B3346696432460120CDE900584AF075
:104010001001B84700B1092420460DF5727DBDE8B6
:10402000F087BAF1070FF6D12046296CFFF776FF2B
:1040300003A800F093FB00BF406C7047F0B54FF051
:10404000FF37CB6BF9B00B6401AC01F1040C0E46E9
:104050000546BCE80F000FC4BCE80F000FC4BCE865
:104060000F000FC49CE80F0084E80F00009706E0E3
:104070006A4629462B6998470828044608D12846ED
:104080001099FFF7C7FE0028F2D0092079B0F0BDE3
:104090006846FFF70FFF062CF7D131462846FFF799
:1040A0003FFF00BF10B414468461DC6BC160002286
:1040B0001C64194610BC53E770B54369C6680B64AD
:1040C000AEB90A46036904460D46014602209847E8
:1040D000072805D008280FD129462046FFF720FFE2
:1040E0003046296CFFF71AFF281D00F037FB01222C
:1040F000FFF736FFFEF7E6F8FEF7E4F8C2682AB1EC
:10410000D1F83CC00022C1F840C029E796E700BFC3
:10411000704700BF836801460BB101201847704704
:10412000012912D009D873B90F2A0CD800EB8200EC
:1041300042681846009B1A6070470339012994BFF2
:10414000012002207047022070470846704700BFD8
:10415000002300B585B00A4603A900911946FFF770
:10416000DFFF039805B05DF804FB00BF012912D002
:1041700009D873B90F2A0CD8009900EB820209689C
:104180001846516070470339012994BF012002206D
:104190007047022070470846704700BF002310B5E3
:1041A00084B003AC039200940A461946FFF7DEFF81
:1041B00004B010BD70B54FF0FF36D36BADF50E7D7A
:1041C00013640DF15C0E02F1040C05460C46BCE8CC
:1041D0000F00AEE80F00BCE80F00AEE80F00BCE82F
:1041E0000F00AEE80F009CE80F008EE80F00169657
:1041F00012E00C2116A86A46FFF7D0FF214616A848
:10420000A84778B969460820049B16AA984705284C
:10421000064608D0092805D068462699FFF7FAFD1A
:104220000028E6D0092616A8FFF744FE30460DF513
:104230000E7D70BD2DE9F04F1E46CC6C89B054F850
:10424000043B0D46174600F003080694002E79D073
:1042500002228DF81C201A0C8DF81D201B04D2B2EE
:10426000059304EB82042B6DB8F1020F08BFAC6B11
:1042700013F001030CD0384605A900F071FB18B902
:10428000082009B0BDE8F08F092009B0BDE8F08F23
:10429000D4F800A0BAF1000FEDD0019300F00803AC
:1042A0000293022E4AD0B4F800A0B4F8029004346D
:1042B000AA6C0F21384629F0010B9344FFF748FF01
:1042C000834539D82AF001025A44824294BF002023
:1042D00001204FEA490303F002030AF0010A43EA0E
:1042E0000A03012B49D0022B32D0002BCCD1B8F1DC
:1042F000000F02D0002840F0CE800434D4F800A093
:10430000BAF1000FCDD1384605A900F029FB0028ED
:10431000BAD1019B002BB3D00F213846FFF718FF0D
:104320000E2102463846FFF739FF38460F216A4A08
:10433000FFF734FF0720A8E70020CAE7D4F804906D
:104340000834B5E71B0205930323ADF81C308AE758
:10435000236823F0004BB8F1000F45D128B1029A31
:10436000002A5CD0BBF1000F74D0002B00DA0434BB
:104370000BF1010B04EB8B04C0E7B8F1000F19D16E
:10438000B0B163682268991C4FEAD2723FF47CAFE7
:1043900005F158010133049100F09180201DFFF7D1
:1043A000B7FD04AB01462846AFF3008000285CD17E
:1043B0000834A3E70D213846D5F82090FFF7C8FE52
:1043C0008145F5D1AB6A9C42F2D12046FFF7D4FC7F
:1043D0000F2102463846FFF7E1FE38462A46002103
:1043E000FFF7DCFE072050E70D213846D5F8209076
:1043F000FFF7AEFE814501D02368B6E7AB6A9C4269
:10440000FAD104230022C5E90B23E318C5F828B02C
:104410006B632368002B5ADB01230193A8E705F1A6
:104420005803CDF80C809146B04604F1040A1E46AC
:104430000EE050460496FFF76BFD0022014604ABE8
:10444000284609F101090AF1040AAFF30080E8B92E
:10445000D945EED10D213846FFF77AFE0346049A7E
:104460000620C5E909242B620FE781460D21384655
:10447000FFF76EFEB9F1020F286225D12B46049A90
:1044800043F82C2F6B620620AC62FEE6464623689A
:10449000DDF80C8069E72046FFF76EFC0246043425
:1044A000AC6328461446AFF3008000283FF4ECAE1E
:1044B000384622460F21FFF771FE0720E5E60D2161
:1044C0003846FFF745FE2862049B6B62DBE70BF181
:1044D000010004EB800079E7000000000023A9E65A
:1044E0000123A7E60223A5E62DE9F043064615467B
:1044F0001C46C3B0042900F2B880DFE801F09C56E6
:10450000B62D0300002C40F0B080102A00F2AD80E0
:104510000368D80600F1F18020AF384600F090F92A
:10452000012438460023B16B04FA03F22A4203F156
:10453000010305D00A4652F804CB1146C0F800C06A
:10454000042B00F10400EFD13846B16300F06EF99E
:10455000002043B0BDE8F083032C40F0868094B285
:1045600004EB1243102B4FEA12457ED803681F0755
:1045700000F1CB8020AF384600F036F9B26B07EB84
:10458000C50154B10B4601EBC401D01AE4001D581B
:1045900043F8045B8B42FAD122443846B26300F000
:1045A00001F9002043B0BDE8F083012C4FEA124826
:1045B00095B256D0052C58D108EB0509B9F1200F5A
:1045C00053D8B8F10F0F73D9A946002D40F084805D
:1045D000B36B65B320AF4FF0000907EBC807043F8A
:1045E00003EBC50553F8041BAB4247F8041FF9D190
:1045F000B9F1000F0FD06F464146102938BF102186
:1046000007EBC101843903EBC90553F8040BAB4236
:1046100041F8040FF9D1012C7FD0B8F10F0FB56329
:1046200042D9B9F1000F02D0684600F0B3F800207B
:1046300043B0BDE8F083C4B923460124826B371D23
:10464000A8B204FA03F101421CBF52F8041B47F858
:1046500023100133102BF4D115F40050E7D1B263CD
:1046600004E008EB0503102B03D9022043B0BDE89A
:10467000F083B8F10F0FF8D83368DA0706D5304663
:1046800023F0030340F8483B00F078F820AF3846A9
:1046900000F074F8B36B002D9DD11D4604353846EB
:1046A000B56300F067F8C2E720A800F06BF8B8E740
:1046B000B9F1100F3FD9A9F110093368D90708D50E
:1046C000304623F0010343F0020340F8483B00F07A
:1046D0005DF8B9F1000F31D033685A071FD4B8F133
:1046E0000F0F24D96F46C8F11005384600F056F870
:1046F000002DB36B80DD20AF6FE723F01003336034
:1047000006F5E87000F09CF806E723F00803036064
:1047100000F5A87000F068F82CE720AFBEE730463F
:1047200023F0040340F8D03B00F038F8D7E720A886
:1047300000F02CF8D6E74FF00009BEE7B8F10F0FF4
:104740003FF646AF20AF384600F020F8B36B002D9F
:104750007FF441AF384600F015F868E700F1340106
:1047600091E838009C46A6464CF8045D90E8FF0F9F
:10477000E54600BD90EC210B704700BF80EC210B9B
:10478000704700BF90EC200B704700BF80EC200BFF
:10479000704700BFD0EC200B704700BFC0EC200B6F
:1047A000704700BFF0EC0201F0EC0211F0EC0221C6
:1047B000F0EC0231F0EC0241F0EC0251F0EC02615D
:1047C000F0EC0271F0EC0281F0EC0291F0EC02A14D
:1047D000F0EC02B1F0EC02C1F0EC02D1F0EC02E13D
:1047E000F0EC02F1704700BFE0EC0201E0EC0211D6
:1047F000E0EC0221E0EC0231E0EC0241E0EC02519D
:10480000E0EC0261E0EC0271E0EC0281E0EC02918C
:10481000E0EC02A1E0EC02B1E0EC02C1E0EC02D17C
:10482000E0EC02E1E0EC02F1704700BFB0FC018176
:10483000B0FC0191B0FC01A1B0FC01B1704700BF18
:10484000A0FC0181A0FC0191A0FC01A1A0FC01B190
:10485000704700BFEC4600B52DE900502DE9FF1F61
:104860004FF000032DE90C0001A9FFF7E7FBDDF88D
:1048700040E012B0704700BFEC4600B52DE9005093
:104880002DE9FF1F4FF000032DE90C0001A9FFF7F0
:1048900013FCDDF840E012B0704700BFEC4600B5F5
:1048A0002DE900502DE9FF1F4FF000032DE90C000A
:1048B00001A9FFF723FCDDF840E012B0704700BF0C
:1048C000EC4600B52DE900502DE9FF1F4FF0000325
:1048D0002DE90C0001ABFFF7E5FBDDF840E012B07D
:1048E000704700BFEC4600B52DE900502DE9FF1FD1
:1048F0004FF000032DE90C0001AAFFF75BFCDDF887
:1049000040E012B0704700BF027A03467AB9427A9B
:10491000A2B14FF0030C4168013A427208680A1DC7
:104920005A60020283F808C0000E1A6070470068DF
:10493000013A1A7202021A60000E7047B0207047E6
:10494000002300B585B003A900910C221946FFF79A
:10495000E7FB039805B05DF804FB00BFF0E700BF7C
:104960002DE9F0434FF0000805460E4685B030466D
:10497000FFF7CAFFB028044600F0BA80070620D52A
:1049800000F0F003802B4DD0902B36D0A02B60D0C0
:10499000B02B73D0C02B00F08A8000F0F803D02B2E
:1049A0000BD100F00702013205230121284642F411
:1049B0000022FFF799FD0028D9D0092005B0BDE8F5
:1049C000F0838300DBB21F1D00230DF10C09194693
:1049D0000D222846CDF80090FFF7A2FB039B60064E
:1049E0004CBFDF1BFF1800230D2228461946CDF8C7
:1049F00000900397FFF7BAFBB9E700F00D030D2B0A
:104A0000DBD0002303AF194600F00F0200972846C1
:104A1000FFF786FB00230D22284619460097FFF773
:104A2000A5FBA4E73046FFF76FFF24022043B0F553
:104A3000004FC2D00023040119462846A2B2FFF756
:104A400053FD0028B9D114F4004F18BF4FF00108EE
:104A50008DE7C3434FF47F6203F007031A4100233D
:104A6000010702F47F6248BF42F48042284619469B
:104A7000FFF73AFD00283FF47AAF9EE7B1283CD01B
:104A8000B22800F0B080B3284AD000F0FC03B42B69
:104A900093D0012300F007021A442846194642F435
:104AA0000022FFF721FD00283FF461AF85E7C6280B
:104AB0004FD0C72861D000F0F803C02B70D0C828B1
:104AC0007CD0C9287FF479AF3046FFF71DFF05235E
:104AD000024601212846140302F00F0204F4702458
:104AE0000A442243FFF700FD00283FF440AF64E78B
:104AF000B8F1000F1CD0002060E73046FFF704FF3C
:104B0000024600283FF459AF10F0F0037FF455AF90
:104B100019462846FFF7E8FC00283FF428AF4CE789
:104B20003046FFF7F1FE0123024619462846D2E738
:104B300003AC43460E22414628460094FFF7F0FAA4
:104B400043460F22284641460094FFF70FFB40469C
:104B500034E73046FFF7D8FE02460323140302F081
:104B60000F0204F470240132284619462243FFF74D
:104B7000BBFC00283FF4FBAE1FE73046FFF7C4FE46
:104B8000024600283FF419AF10F0F0037FF415AF90
:104B900004212846FFF7A8FC00283FF4E8AE0CE704
:104BA000032300F00F0201322846194642F4202266
:104BB000FFF79AFC00283FF4DAAEFEE63046FFF736
:104BC000A3FE0246012102F0F00402F00F021034AD
:104BD0000A440523284642EA0432FFF785FC0028F0
:104BE0003FF4C5AEE9E600230DF10C090D2219468C
:104BF0002846CDF80090FFF793FA3046FFF784FE81
:104C000002064FF002040CD5039B00F07F00A04089
:104C1000184403903046FFF777FE030604F10704BB
:104C2000F2D4039B00F07F02A24003F501731A4403
:104C30000023039228460D221946CDF80090FFF775
:104C400095FA94E60B464FF0030C00B5C26C18467B
:104C5000536885B00832029201A91A0E1B028DF822
:104C60000CC001938DF80D20FFF77AFE05B05DF8BA
:104C700004FB00BF08B5FFF771FE806C08BD00BFE4
:104C800008B5FFF76BFEC06CC379023300EB8300FD
:104C900008BD00BF0A44914200F1FF3300D17047C4
:104CA00010B511F8014B914203F8014FF9D110BD35
:104CB00003460244934200D1704703F8011BF9E711
:104CC0000EB46FF0004100B59CB01DAB0290069091
:104CD000079104910848094953F8042B059100688D
:104CE00002A9019300F08AF80022029B1A701CB0FE
:104CF0005DF804EB03B07047580000200802FFFF86
:104D0000034611F8012B03F8012B002AF9D1704753
:104D1000034613F8012B002AFBD1181A01387047FB
:104D2000034610B5013932B111F8014F013A03F8C9
:104D3000014B002CF7D100211A44934200D110BD41
:104D400003F8011BF9E72DE9F0478E6882469E4281
:104D50000C4690461F4638D88A8912F4906F32D09C
:104D6000256809690133A5EB010965694B4405EB29
:104D7000450505EBD5756D109D4238BF1D465305A1
:104D800031D5294600F060FB064650B90C234FF0A0
:104D9000FF30CAF80030A38943F04003A381BDE887
:104DA000F0874A462169FFF775FFA38923F49063D2
:104DB00043F08003A38126614E4426603E46656130
:104DC000A5EB0905A560BE4200D93E4632464146E4
:104DD000206800F0B7FAA36800209B1BA36023683B
:104DE00033442360DBE72A4600F0A2FB0646002896
:104DF000E1D15046216900F0BFFAC7E72DE9F04F35
:104E000098468B8907461B060D4614469DB00ED565
:104E10000B6963B9402100F017FB2860286120B9B5
:104E20000C233B604FF0FF30D1E040236B61002347
:104E3000099320238DF8293030234FF00109CDF854
:104E40000C80DFF8A4818DF82A3023469A4613F8A7
:104E5000012B0AB1252AF9D1BAEB040B0BD05B4622
:104E6000224629463846FFF76EFF013000F0AA803F
:104E7000099A5A4409929AF80030002B00F0A28057
:104E800000234FF0FF32CDE905230AF1010A049314
:104E900007938DF853301A935446052214F8011BDA
:104EA000514800F041FA049AD8B9D00644BF2023F3
:104EB0008DF85330110744BF2B238DF853309AF8E7
:104EC00000302A2B15D0544600204FF00A0C079AC8
:104ED000214611F8013B303B092B4ED9B0B1079266
:104EE00014E0A0EB080309FA03F31343A24604936A
:104EF000D2E7039B191D1B680391002BBBBF5B42CC
:104F000042F0020207930793B8BF049223782E2B36
:104F10000CD163782A2B35D1039B02341A1D1B68F0
:104F20000392002BB8BF4FF0FF330593DFF8BCA00E
:104F300003225046217800F0F7F940B14023A0EB5E
:104F40000A0003FA00F0049B01340343049314F8AD
:104F5000011B062226488DF8281000F0E5F90028EC
:104F600038D0244B1BBB039B073323F007030833C4
:104F70000393099B3344099367E70C4601200CFB1C
:104F80000232A5E700234FF00A0C194601340593BD
:104F9000204610F8012B303A092A03D9002BC5D03E
:104FA0000591C3E7044601230CFB0121F0E703ABA5
:104FB00000932A463846104B04A9AFF30080421CE8
:104FC0000646D6D1AB895B063FF52CAF09981DB0DC
:104FD000BDE8F08F03AB00932A463846064B04A980
:104FE00000F07CF8EBE700BF7F5800088558000808
:104FF0008958000800000000474D00082DE9F047DF
:10500000164699468A680B6907469342B8BF13460D
:10501000336091F843200C46DDF820800AB101335B
:1050200033602368990642BF3368023333602568D2
:1050300015F0060506D104F1190AE36832689B1AD7
:10504000AB4228DC94F84320131E226818BF0123CA
:1050500092062DD44946384604F14302C047013038
:1050600020D02368E56803F00603042B18BF002551
:1050700032684FF00006A36808BFAD1A226908BF66
:1050800025EAE5759342C4BF9B1AED181A34B54260
:105090001AD1002008E00123524649463846C0474D
:1050A000013003D14FF0FF30BDE8F0870135C4E790
:1050B0003020E11881F843005A1C94F8451022442E
:1050C000023382F84310C5E7012322464946384699
:1050D000C0470130E6D00136D9E700002DE9FF478F
:1050E0000F7E9146782F80460C469A460C9D01F122
:1050F000430207D8622F0AD8002F00F0D980582F1A
:1051000000F0A48004F1420584F842703AE0A7F16F
:105110006303152BF6D801A151F823F0755100084F
:105120008951000805510008055100080551000883
:105130000551000889510008055100080551000873
:10514000055100080551000897520008B9510008A0
:10515000795200080551000805510008B9520008AD
:1051600005510008B9510008055100080551000813
:10517000815200082B681A1D1B682A6004F1420541
:1051800084F842300123A4E020682968060601F172
:1051900004030AD50E682B60002E03DA2D23764215
:1051A00084F843300A235E4819E00E6810F0400F7F
:1051B0002B6018BF36B2EFE72B682068191D2960F5
:1051C000010601D51E6802E04606FBD51E886F2F3A
:1051D0000CBF08230A235248002184F84310656855
:1051E000002DA8BF2168A560A4BF21F004012160A3
:1051F0000EB9002D4DD01546B6FBF3F103FB116738
:10520000C75D05F8017D3746BB420E46F4D9082B31
:105210000BD12368DE0708D5236961689942DEBF98
:10522000302305F8013C05F1FF35521B22614B4646
:1052300021464046CDF800A003AAFFF7DFFE01306B
:105240004CD14FF0FF3004B0BDE8F087344881F80E
:1052500045702968236851F8046B29601D0614D530
:10526000DF0744BF43F0200323601EB9236823F007
:10527000200323601023AFE7236843F0200323605B
:105280007823284884F84530E3E7590648BFB6B28A
:10529000E6E71546BBE72B682668181D616928609C
:1052A00035061B6801D5196002E07006FBD5198030
:1052B000002315462361BAE72B6800211A1D2A60D6
:1052C0001D686268284600F02FF808B1401B606036
:1052D00063682361002384F84330A8E72A464946DF
:1052E00040462369D0470130ABD023689B0713D4D5
:1052F000E068039B9842B8BF1846A4E701233246F2
:1053000049464046D04701309BD00135E3680399B8
:105310005B1AAB42F2DCEBE7002504F11906F5E776
:1053200090580008A1580008034610B5C9B20244BD
:105330009342184601D1002003E0047801338C42E7
:10534000F6D110BD884210B501EB020402D98442A7
:10535000234607D8431EA14208D011F8012B03F8B9
:10536000012FF8E7014602448A4200D110BD13F82C
:10537000014D02F8014DF7E738B50546002940D048
:1053800051F8043C0C1F002BB8BFE41800F010F9D2
:105390001C4A136833B9636014602846BDE838407E
:1053A00000F00CB9A34208D9206821188B4201BF34
:1053B00019685B6809182160EDE71A465B680BB154
:1053C000A342FAD911685018A0420BD120680144B9
:1053D000501883421160E0D118685B680144116085
:1053E0005360DAE702D90C232B60D6E72068211836
:1053F0008B4201BF19685B680918216063605460C3
:10540000CBE738BD5004002070B50E4E0C46316815
:10541000054611B900F0BCF830602146284600F07E
:10542000B7F8431C0AD0C41C24F00304A04207D0E0
:10543000211A284600F0ACF8013001D14FF0FF34BA
:10544000204670BD540400202DE9F041CD1C25F00C
:10545000030508350C2D38BF0C25002D074601DB50
:10546000A94205D90C2300263B603046BDE8F081F7
:105470002E4E00F09DF833681C4634BB2946384652
:10548000FFF7C2FF431C04464DD134682646002E68
:1054900040D123683146384604EB030800F078F821
:1054A00080453AD1216803356D1A25F0030508358A
:1054B0000C2D38BF0C2538462946FFF7A5FF0130D3
:1054C0002BD023682B4423600EE02268521B1ED48D
:1054D0000B2A16D96119A342256018BF5960636869
:1054E00008BF316062514B60384604F10B0600F092
:1054F00065F826F00706231DF21AB6D09B1BA350B1
:10550000B3E76268A3420CBF32605A60ECE72346FF
:105510006468B2E734467668B9E70C2338463B60E6
:1055200000F04CF8A1E72560DEE700BF5004002042
:105530002DE9F041804614460E4621B91146BDE8DA
:10554000F041FFF781BF2AB9FFF716FF254628462D
:10555000BDE8F08100F038F88442074602D8B4EB89
:10556000500F12D821464046FFF76EFF054600282F
:10557000EDD0BC422246314628BF3A46FFF78AFBAF
:1055800031464046FFF7F8FEE1E73546DFE7000029
:1055900038B50023054D044608462B60FCF784FE11
:1055A000431C02D12B6803B1236038BD580400208E
:1055B000014800F011B800BF5C040020014800F071
:1055C0000CB800BF5C04002051F8043C181F002BED
:1055D000BCBF0B58C0187047704770472424242460
:1055E00025732C25640000002C253032753A2530B7
:1055F00032753A25303275002C257325752E2530ED
:10560000346C752C257325752E2530346C7500008F
:105610002C256C64000000002C2573002C256400F0
:105620002C25642E25303264000000002C25642CCB
:1056300025642C25303278002A253034580A0000A1
:1056400044452046364B484B0000000020494E2080
:1056500025730000202B00002D2D2D2D2D00000086
:105660002E2D2D2D2D0000002E2E2D2D2D00000075
:105670002E2E2E2D2D0000002E2E2E2E2D00000061
:105680002E2E2E2E2E0000002D2E2E2E2E0000004F
:105690002D2D2E2E2E0000002D2D2D2E2E00000043
:1056A0002D2D2D2D2E0000002E2D00002D2E2E2E06
:1056B000000000002D2E2D2E000000002D2E2E00AB
:1056C0002E2E2D2E000000002D2D2E002E2E2E2EE3
:1056D000000000002E2E00002E2D2D2D00000000B9
:1056E0002D2E2D002E2D2E2E000000002D2D000021
:1056F0002D2E00002D2D2D002E2D2D2E0000000012
:105700002D2D2E2D000000002E2D2E002E2E2E00D1
:105710002E2E2D002E2E2E2D000000002E2D2D00C1
:105720002D2E2E2D000000002D2E2D2D000000000E
:105730002D2D2E2E00000000A8560008AC560008A3
:10574000B4560008BC560008A4560008C05600080D
:10575000C8560008CC560008D4560008D856000891
:10576000E0560008E4560008EC560008F056000821
:10577000F4560008F85600080057000808570008BB
:105780000C5700085C560008105700081457000812
:105790001C570008205700082857000830570008F9
:1057A00058560008605600086856000870560008F1
:1057B0007856000880560008885600089056000861
:1057C00098560008A05600082D2E2E2D2E00000001
:1057D0002D2E2E2E2D0000002E2D2E2D2E2D0000D4
:1057E0002D2D2E2E2D2D00002E2E2D2D2E2E000097
:1057F0002E2D2E2D2E0000002E2D2D2E2D2E002D87
:105800002E00000046364B484B00000057494445E7
:10581000312D312C57494445322D310041505A51D8
:10582000415000003A544553543132333435363701
:10583000383930002125303264253032642E25304D
:1058400032752563256325303364253032752E2566
:10585000303275256325632F413D2530366C642F2A
:10586000502564532564542564562564257300002F
:10587000205273343120747261636B65722100238E
:105880002D302B2000686C4C00656667454647004C
:105890003031323334353637383941424344454666
:1058A00000303132333435363738396162636465FC
:0258B000660090
:1058B40008B10181B0B000840000000008B101818A
:0858C400B0B0008400000000F8
:1058CC005CD1FF7FB0B0AE801CD2FF7FAB08B18043
:1058DC0034D3FF7F01000000F8D3FF7FB0AA038010
:1058EC0028D4FF7F0100000018D5FF7FB0AF0280E5
:1058FC00C8D5FF7FB0B0A88018D6FF7FB0A80380B2
:10590C0044D6FF7F0100000054D6FF7F03AC2D80EE
:10591C0058D8FF7F01000000F0E4FF7FB0A902809F
:10592C0088E5FF7FB0B0A880D8E5FF7F01000000BC
:10593C00E4E5FF7FB0B0AA801CE6FF7FAE71B280B9
:10594C00ECE6FF7F01000000E8E6FF7FAB3F38800C
:10595C0048E7FF7F0100000054E7FF7FB0B0AA804A
:10596C0090E7FF7F0100000040E8FF7FAA0DB280A6
:10597C00B8E8FF7FB0AF088058EBFF7F0100000054
:10598C005CEBFF7FAD3F0280C8EDFF7F01000000A4
:10599C00A4EFFF7F00840480B8EFFF7F01000000BC
:1059AC00B4EFFF7FB0AD048090F2FF7F00840480E1
:1059BC00B8F2FF7FF4FEFF7FBCF2FF7FF8FEFF7FA3
:0859CC00C8F2FF7F010000009A
:1059D400D0070000010000000A00000046364B48D2
:1059E4004B0000000000000000000000AB120000AB
:1059F400C8AF00004E00000020527334312074728E
:105A040061636B657221000000000000000000006B
:105A1400000000000000000001020304010203046E
:105A240006070809020406085C00002000000000C4
:105A34000000000000000000000000000000000062
:105A44000000000000000000000000000000000052
:105A54000000000000000000000000000000000042
:105A64000000000000000000000000000000000032
:105A74000000000000000000000000000000000022
:0C5A840000000000000000000000000016
:0400000508000000EF
:00000001FF
